:100000000C942A000C9446000C9446000C94460074
:100010000C946F020C942A030C94D0020C94FD02F1
:100020000C9442020C94CE010C9446000C944600B1
:100030000C9446000C9446000C9446000C94460028
:100040000C9446000C9446000000000003000600DB
:1000500008000A0011241FBE20E0A89521BD20E061
:1000600025BFE6EAF7E0A0E6B0E020E002C0059098
:100070000D92A036B207D9F7A0E6B0E020E001C0AB
:100080001D92A238B207E1F70C9449000C94480085
:100090001895CFE5D4E0DEBFCDBF8FE081BB8FEFF9
:1000A00082BB0E947900909884EF91E00E94EE005C
:1000B000909A84EF91E00E94EE00F5CFFFCF039677
:1000C00065E070E00E948203CB01AA27BB2723E0F2
:1000D000880F991FAA1FBB1F2A95D1F720E030E097
:1000E0002817390728F42F5F3F4F28173907D8F30F
:1000F0000895CF93C0E08C2F0E94E300CF5FC730FC
:10010000D0F30E948A000E94A3000E94AD00789460
:10011000CF91089582E00E94C60012BE81E009B628
:10012000082A09BE10926E0010926F0010927000A3
:100130001092710010927A0010927B0010927C0055
:1001400010927D00089583E00E94CC001DBC1CBC71
:1001500084E009B6082A09BE089583E00E94D2000F
:1001600014BC80E409B6082A09BE109276001092E9
:10017000770010927800109279001092720010921D
:10018000730010927400109275000895982F83B731
:10019000887F892B83BF0895982F8EB5887F892B00
:1001A0008EBD0895982F85B5887F892B85BD0895CC
:1001B000873040F4E82FFF27EE0FFF1FE05AFF4F74
:1001C000608371830895873040F4E82FFF27EE0F96
:1001D000FF1FE05AFF4F108211820895EF92FF92A5
:1001E0000F931F93AC0183B7E82FFF27EE0FFF1F7C
:1001F000E85BFF4F249180E091E07A01002711270E
:1002000002C0880F991F2A95E2F79C0144275527C1
:1002100060E072E18AE790E00E949603C801B701AE
:100220000E946303DC01CB01BC01CD0128EE33E069
:1002300040E050E00E94960310927E0010927F00F2
:10024000109280001092810080917E0090917F003A
:10025000A0918000B091810082179307A407B50791
:1002600098F31F910F91FF90EF90089510926E00F8
:1002700010926F00109270001092710010927A002C
:1002800010927B0010927C0010927D000895809166
:100290006E0090916F00A0917000B0917100BC0150
:1002A000CD01089510927600109277001092780098
:1002B00010927900109272001092730010927400E4
:1002C0001092750008958091760090917700A0912A
:1002D0007800B0917900BC01CD0108958930A1F07A
:1002E0008A3049F08DEF0FB408220FBC81E00FB4C3
:1002F000082A0FBC11C082E00FB4082A0FBC81E0AD
:100300000FB4082A0FBC08C082E00FB4082A0FBC43
:100310008EEF0FB408220FBC88E00EB4082A0EBC82
:1003200080E80FB4082A0FBC8FEB0FB408220FBC73
:1003300080E20FB4082A0FBC8FEE0FB408220FBC66
:100340001BBC1ABC19BC18BC08958DEF0FB4082251
:100350000FBC8EEF0FB408220FBC87EF0EB408223B
:100360000EBC8FE70FB408220FBC8FEB0FB408222E
:100370000FBC8FED0FB408220FBC8FEE0FB4082214
:100380000FBC08959C01832F99278BBD2ABD08952A
:100390009C01832F992789BD28BD08951F920F9234
:1003A0000FB60F9211242F933F934F935F936F9348
:1003B0007F938F939F93AF93BF93EF93FF9380911E
:1003C0006E0090916F00A0917000B0917100019645
:1003D000A11DB11D80936E0090936F00A0937000DB
:1003E000B093710080916E0090916F00A0917000A9
:1003F000B09171000097A105B105F9F080917E00E0
:1004000090917F00A0918000B09181000196A11D84
:10041000B11D80937E0090937F00A0938000B093E5
:1004200081008091600090916100892BD1F0E09172
:100430006000F0916100099514C080917A0090915C
:100440007B00A0917C00B0917D000196A11DB11DA3
:1004500080937A0090937B00A0937C00B0937D0002
:10046000CDCFFF91EF91BF91AF919F918F917F91F0
:100470006F915F914F913F912F910F900FBE0F9011
:100480001F9018951F920F920FB60F9211242F9361
:100490003F934F935F936F937F938F939F93AF930C
:1004A000BF93EF93FF938091620090916300892B3B
:1004B00029F0E0916200F09163000995FF91EF91BE
:1004C000BF91AF919F918F917F916F915F914F916C
:1004D0003F912F910F900FBE0F901F9018951F9274
:1004E0000F920FB60F9211242F933F934F935F9368
:1004F0006F937F938F939F93AF93BF93EF93FF93EC
:100500008091760090917700A0917800B091790069
:100510000196A11DB11D8093760090937700A09362
:100520007800B09379008091760090917700A09147
:100530007800B09179000097A105B10561F0809134
:100540006A0090916B00892BD1F0E0916A00F091E4
:100550006B00099514C08091720090917300A09176
:100560007400B09175000196A11DB11D80937200B9
:1005700090937300A0937400B0937500E0CFFF9147
:10058000EF91BF91AF919F918F917F916F915F910B
:100590004F913F912F910F900FBE0F901F90189584
:1005A0001F920F920FB60F9211242F933F934F93E8
:1005B0005F936F937F938F939F93AF93BF93EF93CB
:1005C000FF938091640090916500892B29F0E09160
:1005D0006400F09165000995FF91EF91BF91AF9193
:1005E0009F918F917F916F915F914F913F912F914B
:1005F0000F900FBE0F901F9018951F920F920FB67D
:100600000F9211242F933F934F935F936F937F9398
:100610008F939F93AF93BF93EF93FF938091660067
:1006200090916700892B29F0E0916600F0916700B6
:100630000995FF91EF91BF91AF919F918F917F911C
:100640006F915F914F913F912F910F900FBE0F903F
:100650001F9018951F920F920FB60F9211242F938F
:100660003F934F935F936F937F938F939F93AF933A
:10067000BF93EF93FF938091680090916900892B5D
:1006800029F0E0916800F09169000995FF91EF91E0
:10069000BF91AF919F918F917F916F915F914F919A
:1006A0003F912F910F900FBE0F901F90189588E0EB
:1006B00002B4082A02BC089580E809B6082A09BED7
:1006C000089583BD0895629FD001739FF001829FBA
:1006D000E00DF11D649FE00DF11D929FF00D839FD1
:1006E000F00D749FF00D659FF00D9927729FB00D6E
:1006F000E11DF91F639FB00DE11DF91FBD01CF0181
:1007000011240895AA1BBB1B51E107C0AA1FBB1FE0
:10071000A617B70710F0A61BB70B881F991F5A958D
:10072000A9F780959095BC01CD01089597FB092EFE
:1007300005260ED057FD04D014D00AD0001C38F482
:1007400050954095309521953F4F4F4F5F4F0895FD
:10075000F6F790958095709561957F4F8F4F9F4FDD
:100760000895A1E21A2EAA1BBB1BFD010DC0AA1FF2
:10077000BB1FEE1FFF1FA217B307E407F50720F00A
:10078000A21BB30BE40BF50B661F771F881F991F85
:100790001A9469F760957095809590959B01AC01CE
:0607A000BD01CF01089528
:00000001FF
